:020000040000FA
:0400000000EF7CF0A1
:04F7FC000000000009
:10F80000AFEF7FF000C0E5FF01C0E5FF00EE62F062
:10F8100006EC7FF0006E00C0F3F000C0F4F006ECE0
:10F820007FF0006E0001E96F00500001F42706EC44
:10F830007FF0006E0001E86F00500001F42706EC35
:10F840007FF0006E00C0F5F000500001F4270001C9
:10F85000F551040A24E10001E951D8A4DBD0E851B4
:10F86000D8A4D8D00001F351020A01E0D3D006ECAD
:10F870007FF0006E0001EB6F00500001F42706ECF2
:10F880007FF0006E0001EA6F00500001F42706ECE3
:10F890007FF0006E0001F427F451D8A4B3D000012A
:10F8A000F551010A20E106EC7FF0006E0001F4271B
:10F8B000F451D8A4A7D00001F2B3B9EC7DF08FECDD
:10F8C0007FF00001F2A50BD0C00E0001E46FF70E2F
:10F8D000E56FE66BE76BB9EC7DF08FEC7FF0590ECE
:10F8E00074EC7FF09AD00001EB510001E71914E1AC
:10F8F0000001EA510001E6190FE10001E9510001A0
:10F90000E5190AE1C00E0001E815006EC00E000105
:10F91000E415016E00180FE00001F2A302D0B9EC6B
:10F920007DF08FEC7FF0E8C0E4F0E9C0E5F0EAC0DC
:10F93000E6F0EBC0E7F00001F551040A01E15ED00A
:10F940000001F551D8A462D00001F351D8B456D0CB
:10F950000001EB51D8A45AD0EA51E00BD8A456D0FC
:10F960000001F2A912D00001F3514EEC7EF0400EDE
:10F97000A5EC7FF00001E9514EEC7EF00001E8516A
:10F980004EEC7EF0200EA5EC7FF0EAC0F8FFE9C057
:10F99000F7FFE8C0F6FF000100EE6AF028EE00F085
:10F9A000E8513F0BD926D8B0DA2ADD5206EC7FF0B9
:10F9B0000001F427DC6E0900F55C05E00001F2832C
:10F9C0002A0EA5EC7FF00001F2A906D0DF504EEC24
:10F9D0007EF0200EA5EC7FF00001F32FE7D706ECB8
:10F9E0007FF0006E0001F427F45108E00001E469A3
:10F9F000E569E669E7690001F29304D0580E74ECFA
:10FA00007FF00BD07A0E74EC7FF007D0750E74EC9B
:10FA10007FF003D06C0E74EC7FF0E4CF01F0E4CF04
:10FA200000F01200FF0E926E936E946E966EDAECFA
:10FA30007FF0970ED56E898A929A766A3F0E756E20
:10FA40007086728A7284728C7290718C718E0001D1
:10FA5000E46BE56BE66BE76B0001E86BE96BEA6B67
:10FA6000EB6B8FEC7FF00001F26B93988A88899A98
:10FA700071984B0EA5EC7FF0B9EC7FF00001EC6BB8
:10FA8000ED6B89BA02D0B9EC7FF00001606BC6EC77
:10FA90007EF000016051D8B45CD0899A71988AA830
:10FAA00002D08A9801D08A8861C000F00050520AC2
:10FAB00003E165EC7FF00BD00050500A03E156ECF7
:10FAC0007FF005D00050560A02E182EC7EF0000182
:10FAD000F2A13FD00050450A03E144EC7FF039D059
:10FAE00000503A0A03E102EC7CF033D00050720A75
:10FAF00003E1A5EC7EF02DD00050410A03E1DDECDE
:10FB00007FF027D00050760A24E1006A000162519C
:10FB1000300A01E1002A0050D880E866D890006AD7
:10FB200000360050010BE838E840F46E0001F25155
:10FB3000F70BF410F26F320E0001625D006A0036BE
:10FB40000050010BE838F46E0001F251EF0BF41095
:10FB5000F26F0001F2B195D70001ED51800F800FD7
:10FB600002E1A10EEC5DD8A08CD7DDEC7FF089D747
:10FB7000120000C0E5FF01C0E5FF02C0E5FF03C0C1
:10FB8000E5FF0001E4513F0B04E0210EA5EC7FF0FE
:10FB90007CD00001E75103E1E651E00BD8A475D019
:10FBA000E4C000F0E5C001F0026A036A0350800F70
:10FBB000800F08E1000E025C05E1F80E015C02E135
:10FBC000000E005C01E361D0E4C000F0E5C001F08C
:10FBD000E6C002F0E7C003F000500110021003106D
:10FBE00013E100C8E0F001C8E1F002C8E2F003C888
:10FBF000E3F00801006BEF0E016F7C0E026FF00E58
:10FC0000036F0001F28515D00050C00A07E10150D2
:10FC1000F70A04E1025002E1035001E00AD0E0C01B
:10FC20003CF8E1C03DF8E2C03EF8E3C03FF8000117
:10FC3000F2950001F2A70BD0200EA5EC7FF0000199
:10FC4000E5514EEC7EF00001E4514EEC7EF0E6C052
:10FC5000F8FFE5C0F7FFE4C0F6FF940EC1EC7FF0BB
:10FC60000A0008EE00F00001080EEE6F080EEF6FBC
:10FC7000EE50F56E0F00EF2FFBD7840E82D9EE2FDA
:10FC8000F5D7A694570E74EC7FF0E4CF03F0E4CFE1
:10FC900002F0E4CF01F0E4CF00F0120000C0E5FF75
:10FCA00001C0E5FF02C0E5FF006E00380F0B026ED9
:10FCB000300E02260250016E3A0E015C06E301503E
:10FCC000026E070E02260250016E0150A5EC7FF075
:10FCD0000F0E0014006E300E00260050016E3A0E1A
:10FCE000015C06E30150006E070E00260050016E15
:10FCF0000150A5EC7FF0E4CF02F0E4CF01F0E4CFB7
:10FD000000F0120000EE62F0000160050001EF6FEC
:10FD1000EF07010EEE6FEE51D4EC7FF004E10A0E16
:10FD2000EE6FD4EC7FF0EE5CD8A41200EE2BEF2F38
:10FD3000F2D7EE51D4EC7FF0D8A41200560E74EC3A
:10FD40007FF00001F281F295120000C0E5FF00EEA5
:10FD500062F006EC7FF0F76E06EC7FF0F66E720E46
:10FD6000A5EC7FF0200EA5EC7FF0100E006E0900D0
:10FD7000F5504EEC7EF0200EA5EC7FF0002EF7D76C
:10FD80000A0EA5EC7FF0E4CF00F01200CEEC7FF07D
:10FD9000000100EE60F0E6EC7EF0E86614D07450EE
:10FDA000EE6EEE6FEF6FD8B40ED0CEEC7FF0E6ECD7
:10FDB0007EF0E86608D07450EE6EEF27EE2FF5D790
:10FDC000EF53D8B412000001606B1200A4BA08D03F
:10FDD000F2A4FCD70001EC2B01E3ED2BE86815D071
:10FDE0008A9871B202D071A404D0B9EC7FF0E868AF
:10FDF0000CD071A009D0745005E1CEEC7FF0E6EC98
:10FE00007EF003D0DDEC7FF0E86A12000001EECF57
:10FE1000EEF0EECFEFF0D00EEE27EF27F60EEE2548
:10FE2000F90ED8B0EE27F60EEF25F90ED8B0EF2771
:10FE3000EE39EF25E850120000EE68F00001605145
:10FE4000F80F0001EE6F09E0F05D07E3EE50A86ED9
:10FE500083EC7FF0A92AEE2FF9D7A86A83EC7FF014
:10FE6000120000C0E5FF01C0E5FF006A00EE62F08D
:10FE7000060E016EEE500026012EFCD70050E4CF96
:10FE800001F0E4CF00F0120000EE61F000016051DB
:10FE90000001EE6F07E0EE0705E0EE50A5EC7FF005
:10FEA000EE2FFBD70A0EA5EC7FF0120031EC7FF0AD
:10FEB000B80A0AE1010EA96E080E0001F06F1CECF1
:10FEC0007FF0500E74EC7FF0120031EC7FF0A00A4E
:10FED0000AE10A0EA96E100E0001F06F1CEC7FF013
:10FEE000520E74EC7FF0120000C0E5FF006E200E91
:10FEF000A5EC7FF00050A5EC7FF00A0EA5EC7FF09A
:10FF0000E4CF00F01200A69EA69CA684550EA76E14
:10FF1000AA0EA76EA682A6B2FED7A6941200000172
:10FF2000F2930001400EEE6F08EE00F0EE68EE2F47
:10FF3000FDD71200700ED36E9B8CFF0E92689368F3
:10FF400094689668626AF19E120000C0E5FF006E38
:10FF5000A4A8FED700C073FFE4CF00F0120017EE94
:10FF6000FFF027EEFFF0F86AA68EA69C12EC7DF05B
:10FF7000FFD772A2FED7898A745074507198718825
:10FF80001200A66E550EA76EAA0EA76EA6821200CC
:10FF9000CAEF7FF012EC7DF0CCEF7FF0F70ED76E5A
:10FFA000F80ED66EF2941200A96EA69CA69EA680AC
:0EFFB000A85012009AEC7FF01200FEEF7BF0DA
:020000040030CA
:0E000000FF38FAE2FF4EBBFFFFFFFFFFFFFFDE
:0200000400F00A
:0400000000000000FC
:00000001FF
